:020000040000FA
:1000000080312628FF3FFF3F80310B1D090045301E
:10001000200095006C08963E8600203003182130A1
:1000200087000108F100EC0A710E30390C38F0003D
:10003000F136F13671082500910070089300200018
:100040006C085A3A0319EC010B110900880183313D
:10005000DB2BD100210065082000D50021006408B9
:100060002000D4002100640A0319650A0319003432
:100070003E28540A0319550A03195A282000550826
:10008000D3005408D2005308C5005208C400FC2015
:1000900080314508D5004408D4005208013ECF0005
:1000A0000030533DD0005506031D582854084F0614
:1000B000031939282100640820005202CF002100D2
:1000C00065082000533BD0004F08013ED6000030A9
:1000D000503DD700D801D9016D08F200F301F401B9
:1000E000F5015908F9005808F8005708F7005608B4
:1000F000F600D72080317508D9007408D80073083D
:10010000D7007208D6004E08860087015608C03F07
:100110005708C13F5808C23F5908C33F210064082F
:10012000FE3E2000D600FF302100653D2000D700B4
:10013000D801D9016D08F200F301F401F501590865
:10014000F9005808F8005708F7005608F600D720BD
:1001500080317508D9007408D8007308D700720878
:10016000D60021004D082000D60721004E082000AF
:10017000D73D0030D83DD93D6608D6076708D73D42
:100180006808D83D6908D93D51088600870156089E
:10019000C03F5708C13F5808C23F5908C33F5508E0
:1001A0002100E500200054082100E4000134A001F2
:1001B000A101A201A301721CE5287608A007770817
:1001C000A13D7808A23D7908A33DF635F70DF80D5D
:1001D000F90DF536F40CF30CF20C75087404730485
:1001E0007204031DDB282308F5002208F40021080F
:1001F000F3002008F200080021004F082000C8008A
:10020000210050082000C900CA01CB016608C807B8
:100210006708C93D6808CA3D6908CB3D4508C8075D
:1002200001300318C9070318CA070318CB0745088C
:10023000CD004408CC00FF30CC05CD01CC35CD0D30
:100240004B08BF004A08BE004908BD004808BC0072
:100250004D08C1004C08C0000230C2004630C30047
:100260008E31012680310038031D3B29FF302000EC
:10027000C400C50008004630F2018F31E927803103
:1002800073082000C5007208C400FF304502F83032
:1002900003194402031C08003629B3001030F20091
:1002A0007E30F3000230F4007608E52181317208D7
:1002B000BE00B401B501B601B7013E0803196729B4
:1002C00033080319C22903303E020318C229103033
:1002D000F2003E30F3000C30F4007608E521813165
:1002E0007308B2007208B1001030F2002F30F30032
:1002F0000330F4007608E52181317208BC0010302B
:10030000F2005030F3000430F4007608E52181312A
:100310007208BD000730BF003F0803199729BD08C8
:1003200003199729BD03BF038C29BC03BF033F08F2
:10033000031DBC08031D95293108013EB80000309B
:10034000323DB900BA01BB013F08031D3818AE2980
:10035000BB36BA0CB90CB80CBF03A4293B08B700D4
:100360003A08B6003908B5003808B4003F083D0225
:100370003C07890ABF29B435B50DB60DB70D890BF9
:10038000BB29DC293E0BDC291030F2003030F300B1
:100390001630F4007608E52181317508B70074083D
:1003A000B6007308B5007208B4000A30B435B50D54
:1003B000B60DB70D890BD6293708F9003608F800B5
:1003C0003508F7003408F6000800A800AF017208ED
:1003D000090709070907AD00A901AA01AB01AC0192
:1003E00073082D02FF3EB000A000A036A036A03654
:1003F0002008AE0030080739073CB0002E08280757
:10040000A000860087010108A100300A082AA13651
:10041000890B072A21080139A200A3012F0A122AF9
:10042000A235A30D890B102A2208A4002308A500D9
:100430000030A51BFF30A600A7002408A90425084A
:10044000AA042608AB042708AC04AF0AF30AF40B8D
:10045000F0292C08F5002B08F4002A08F3002908DD
:10046000F200080020006908680467046604031DA0
:100470000034BE30DC000130DD00BC01BD01BE0136
:10048000BF015D08C1005C08C0001030C2004C30E4
:10049000C3008E3101268231003803190034200058
:1004A00050030319672A5008043A0319672A5008B1
:1004B000063A0319672A50080B3A0319672A5008AD
:1004C0000C3A0319672A50080E3A031DD22A57081E
:1004D000E600E701E801E9015608C400C501C601CC
:1004E000C7016608C8006708C9006808CA0069082B
:1004F000CB004A08CB004908CA004808C900C80117
:1005000044084804E60045084904E70046084A0450
:10051000E80047084B04E9005508C400C501C601BE
:10052000C7016608C8006708C9006808CA006908EA
:10053000CB004A08CB004908CA004808C900C801D6
:1005400044084804E60045084904E70046084A0410
:10055000E80047084B04E9005408C400C501C6017F
:10056000C7016608C8006708C9006808CA006908AA
:10057000CB004A08CB004908CA004808C900C80196
:1005800044084804E60045084904E70046084A04D0
:10059000E80047084B04E9008F3140278231003AD8
:1005A000031D013410302000DC070318DD0A013080
:1005B0005D02FE3003195C02031800343D2A730803
:1005C000AA007208A900A935AA0DA935AA0D6A08C2
:1005D000A9076B08AA3DB001AB01AC01AD01AE01AA
:1005E000AF0180302300950020002A0823009200EC
:1005F00020002908230091008B131514000000002F
:100600008B17230013082000A000230014082000EB
:10061000A100A201A3012B08A4002C08A5002D080D
:10062000A6002E08A7000E30A435A50DA60DA70D17
:10063000890B142B20082404AB0021082504AC00EE
:1006400022082604AD0023082704AE00AF0AA90A39
:100650000319AA0A02302F02031CF12AB008031D55
:10066000332B7408342B7508A800860087012B08EB
:10067000C03F2C08C13F2D08C23F2E08C33F0230A7
:10068000B00A300203180800EC2AF6007208F607D8
:1006900076088600870101082000A000A101A201C0
:1006A000A3017608013E86000108A400A501A60169
:1006B000A7012608A7002508A6002408A500A40174
:1006C0007608023E86000108A800A901AA01AB0134
:1006D0002908AB002808AA00A901A8017608033E52
:1006E00086000108AF00AE01AD01AC012C08A804E2
:1006F0002D08A9042E08AA042F08AB042808A40476
:100700002908A5042A08A6042B08A7042008240405
:10071000F20021082504F30022082604F40023082F
:100720002704F5000800AA004038A4002308A5000B
:100730002208A6002108A7002008A80005300314FD
:10074000F2002430F301B723F900790DA900AA01C2
:100750002A08243E8600870101088E31E82683316D
:1007600020000630AA0A2A0203180800A82BF50068
:10077000F801720878020318D82B78087507F4007E
:10078000860087010108F600F7018030F335730514
:10079000F4007608803974060319D02B0930F3066B
:1007A0000830F635F70A7702031CC52BF80AB92B77
:1007B00073087F39080096308400203085005A3055
:1007C000FE000030FF0084319D248331FB01E601EF
:1007D000E701E801E901EA01EB01EC01ED01CD30AF
:1007E0008400003085001330FE000030FF008431AB
:1007F0009D240130EE002100FF30E000FF30E100D9
:10080000FF30E200FF30E300FF30E400FF30E5009E
:1008100020008831DE28F5018030F2007508963E10
:10082000F300203003182130F400730886007408A8
:100830008700720881005A30F50A7502031C0C2CDF
:1008400004309C001F309B000C3025009300920167
:10085000910121008C12200095010B118B160800CC
:10086000B6003730AB01AC01AD01AE01AF01AF0A4C
:100870008C31F5248431B700B71F402C37080800AD
:1008800037193E2C3508AE003408AD003308AC00F3
:100890003208AB00AF01AF0A36088C31F52C2200CC
:1008A0008C100C1624001B309512F200F20B562C03
:1008B00022001B308C14F200F20B5C2C22001B3047
:1008C0008C10F200F20B622C240095160800F60141
:1008D000F701721C6F2C7408F6077508F73DF435A4
:1008E000F50DF336F20C73087204031D692C7708BA
:1008F000F3007608F2000800F301822C7408FF3A36
:10090000031D8C2CFF308E31E8268431F4008130B9
:10091000F30A7302031C7E2C74080800F200F2082C
:10092000031D952C0A30F300962CF301F4012400EA
:100930001508F03973049500080064008001013146
:100940000130FE020030FF3B7F087E0403190034B3
:100950009E2C0230BC01BD01BE01BF01C001C1001F
:10096000C201C3018E31012E8B122500930121009B
:100970008C1220008C120800FF3FFF3FFF3FFF3F1B
:10098000FF3FFF3FFF3FFF3FFF3FFF3FFF3FFF3F77
:10099000FF3FFF3FFF3FFF3FFF3FFF3FFF3FFF3F67
:1009A000FF3FFF3FFF3FFF3FFF3FFF3FFF3FFF3F57
:1009B000FF3FFF3FFF3FFF3FFF3FFF3FFF3FFF3F47
:100E00000034FF3FFF3FFF3FFF3FFF3FFF3FFF3FFC
:100E1000FF3FFF3FFF3FFF3FFF3FFF3FFF3FFF3FE2
:100E2000FF3FFF3FFF3FFF3FFF3FFF3FFF3FFF3FD2
:100E3000FF3FFF3FFF3FFF3FFF3FFF3FFF3FFF3FC2
:100E4000FF3FFF3FFF3FFF3FFF3FFF3FFF3FFF3FB2
:100E5000FF3FFF3FFF3FFF3FFF3FFF3FFF3FFF3FA2
:100E6000FF3FFF3FFF3FFF3FFF3FFF3FFF3FFF3F92
:100E7000FF3FFF3FFF3FFF3FFF3FFF3FFF3FFF3F82
:100E8000FF3FFF3FFF3FFF3FFF3FFF3FFF3FFF3F72
:100E9000FF3FFF3FFF3FFF3FFF3FFF3FFF3FFF3F62
:100EA000FF3FFF3FFF3FFF3FFF3FFF3FFF3FFF3F52
:100EB000FF3FFF3FFF3FFF3FFF3FFF3FFF3FFF3F42
:100EC000FF3FFF3FFF3FFF3FFF3FFF3FFF3FFF3F32
:100ED000FF3FFF3FFF3FFF3FFF3FFF3FFF3FFF3F22
:100EE000FF3FFF3FFF3FFF3FFF3FFF3FFF3FFF3F12
:100EF000FF3FFF3FFF3FFF3FFF3FFF3FFF3FFF3F02
:100F0000FF3FFF3FFF3FFF3FFF3FFF3FFF3FFF3FF1
:100F1000FF3FFF3FFF3FFF3FFF3FFF3FFF3FFF3FE1
:100F2000FF3FFF3FFF3FFF3FFF3FFF3FFF3FFF3FD1
:100F3000FF3FFF3FFF3FFF3FFF3FFF3FFF3FFF3FC1
:100F4000FF3FFF3FFF3FFF3FFF3FFF3FFF3FFF3FB1
:100F5000FF3FFF3FFF3FFF3FFF3FFF3FFF3FFF3FA1
:100F6000FF3FFF3FFF3FFF3FFF3FFF3FFF3FFF3F91
:100F7000FF3FFF3FFF3FFF3FFF3FFF3FFF3FFF3F81
:100F8000FF3FFF3FFF3FFF3FFF3FFF3FFF3FFF3F71
:100F9000FF3FFF3FFF3FFF3FFF3FFF3FFF3FFF3F61
:100FA000FF3FFF3FFF3FFF3FFF3FFF3FFF3FFF3F51
:100FB000FF3FFF3FFF3FFF3FFF3FFF3FFF3FFF3F41
:100FC000FF3FFF3FFF3FFF3FFF3FFF3FFF3FFF3F31
:100FD000FF3FFF3FFF3FFF3FFF3FFF3FFF3FFF3F21
:100FE000FF3FFF3FFF3FFF3FFF3FFF3FFF3FFF3F11
:100FF000FF3FFF3FFF3FFF3FFF3FFF3FFF3FFF3F01
:10100000FF3FFF3FFF3FB600043E860087013508E3
:10101000BA003408B9003308B8003208B700011824
:1010200018280930B735B80DB90DBA0D890B12283B
:101030003A08AE003908AD003808AC003708AB00FC
:101040001230AF01F5248831BB00BB1F2A28EF30D6
:101050008D220034FF30E82688312000BB00FF3AA3
:1010600003192A283B08FE3A03190134EE302828D8
:1010700020000530CC01CB01CA00F430C900FA30A1
:10108000CD00CE01CF01D001C101C20184310B24BA
:1010900088314208F3004108F2004930F4004D3035
:1010A000F5008231DF228831C10A0319C20A4C08D7
:1010B0004B044A044904031D632850084F044E049E
:1010C0004D040319CE284C08B5004B08B4004A085B
:1010D000B3004908B200DB30032088312000C00093
:1010E000C008031D76280230212288312000C40167
:1010F000C501C601C70150084702031D89284F08D2
:101100004602031D89284E084502031D89284D0803
:1011100044020318CB284708460445044404031935
:101120009528DB30F300D02088312000C801C301AE
:101130004308803A0319BE286E086C0603199828E4
:10114000FF30E82688312000BC00BC36BC36BC36F7
:101150003C08BD006E08963EBE00203003182130CA
:10116000BF003E0886003F0887003D088100EE0A68
:101170006E085A3A0319EE01C30A98280430C80AC7
:101180004802031C9728C40A0319C50A0319C60A92
:101190000319C70A7B28F026883149288431B42CEA
:1011A000FF30E8268831FF30E8268831FF30E82616
:1011B0008831F400FF3A031D0800D6282100F030E2
:1011C000CB01CC01C101C20199001F3098008030D1
:1011D0008B00413022009D00CC3021008C00230088
:1011E0008C0180302100950003301710AF00AC3027
:1011F000AE00B330AD00AD0BFB28AE0BFB28AF0B40
:10120000FB28640015302100AF00DA30AE0020303A
:10121000AD00AD0B0929AE0B0929AF0B0929102927
:101220002000DB300C14292488312100C500C508BA
:10123000031D1D29013021228831FE2388314027DA
:1012400088312100C500C508031D29290630212247
:10125000883121004C082000C50021004B082000E7
:10126000C400B030C600C730C700C630C800C330A5
:10127000C9000A2588310038031956292100CB0AF4
:101280000319CC0A46081239031D29293808573A90
:10129000031D29293908413A031D29293A08563ADC
:1012A000031D2929C10A0319C20A2929210042085C
:1012B0004104031D5E2903302122883121004208A8
:1012C0002000A500210041082000A40097228831B9
:1012D0002908A7002808A60009248831250821002C
:1012E000BC00200024082100BB00CB01CC014C082D
:1012F0002000C50021004B082000C400B030C6000B
:10130000C730C700C630C800C330C9000A258831BD
:1013100000380319A9292100CB0A0319CC0A460871
:101320001239031D77293808573A031D77293908E0
:10133000413A031D77293A08563A031D77290130AF
:10134000BB020030BC3B3B0A03193C0A0319AC2921
:10135000772909302122883121004408F30043080D
:10136000F200042488310038031DB92907302122F6
:101370008831872388315B23CB01CC01C730200023
:10138000CE00BD3080312920883100380319F6297C
:101390004C082000A10021004B082000A0002100E3
:1013A00040082000A50021003F082000A4002100E3
:1013B0003E082000A30021003D082000A2002100DB
:1013C0004A082000A900210049082000A8002100A7
:1013D00048082000A700210047082000A6002A2274
:1013E00088312100CB0A0319CC0ABE294C08200001
:1013F000A10021004B082000A000A201A301A4012C
:10140000A501A601A701A801A9012A228431A924C6
:1014100088313820883175300C10F501F401F30063
:101420003030F200B12388312000DB300C14292445
:1014300088312100C500C508031D5E2901305C29E3
:10144000202AF500FA308D22883175088D228831E6
:101450006300282A2108AF002008AE00AE35AF0D8A
:10146000AE35AF0D6A08AE076B08AF3DB101B108EC
:10147000031D422A2508AD002408AC002308AB0058
:101480002208492A2908AD002808AC002708AB002B
:101490002608AA00B00184302300950020002F0800
:1014A0002300920020002E082300910020002A082B
:1014B000F2002B08F3002C08F4002D08F5000E3084
:1014C000F536F40CF30CF20C890B602A7308230038
:1014D00094007208930055308B139600AA30960042
:1014E0009514000000008B1723009518742A200023
:1014F000B00AAE0A0319AF0A0E30AA35AB0DAC0D17
:10150000AD0D890B7D2A02303002031C4B2A0230BC
:10151000B10A310203180800372AF400F2007B08F0
:1015200049238831FB0A7B08031D0800932AFF30FA
:10153000412388312000B200FE30B301B401B5016F
:10154000412388312000AA00AB01AC01AD01320873
:10155000AE003308AF003408B0003508B1003008E1
:10156000B1002F08B0002E08AF00AE012A082E04EB
:10157000B2002B082F04B3002C083004B4002D084F
:101580003104B500FD30412388312000AA00AB01B1
:10159000AC01AD013208AE003308AF003408B00032
:1015A0003508B1003008B1002F08B0002E08AF0098
:1015B000AE012A082E04B2002B082F04B3002C0819
:1015C0003004B4002D083104B500FC3041238831CB
:1015D0002000AA00AB01AC01AD013208AE00330817
:1015E000AF003408B0003508B1003008B1002F0852
:1015F000B0002E08AF00AE012A082E04B2002B085E
:101600002F04B3002C083004B4002D083104B500B9
:10161000F5003408F4003308F3003208F200DE303D
:10162000F900EC30F800E630F7006D30F60080315C
:10163000D72088310B307207B2000030733DB30001
:101640000030743DB4000030753DB500F200FF304D
:101650004923883120003408F200FE3049238831C4
:1016600020003308F200FD30492388312000320881
:10167000F200FC30492320003508A9003408A800F6
:101680000800F20023009501720891001514130858
:101690000800F300043023009500730891007208DD
:1016A00093008B1355309600AA30960095148B1733
:1016B000951C0800582B20006B08F3006A08F20004
:1016C000F401F501210056087502031D692B550828
:1016D00074020318080094308B13230095007308DC
:1016E00092007208910055309600AA309600951429
:1016F000000000008B172300151A7B2B0830F4071D
:101700000318F50A2030F2070318F30A622B2100B0
:101710000230D501D60001302000EA008530EB0010
:101720006A08F2001F30F205720803199A2B72083A
:10173000203CF20072082100D502031CD603720877
:101740002000EA070318EB0AE0302100D505FF303E
:10175000D6052000EB132100D636D50CD636D50C95
:1017600008000430A501A400A301A201210019086A
:101770002000A00013302100990020008C122100CD
:101780000C082000A100DE3021008C002000123067
:101790000C10A600200025087502031DD92B240873
:1017A0007402031DD92B23087302031DD92B2208B1
:1017B0007202031CEC2B640003142000260D210090
:1017C000970020002208F2022308F33B2408F43B90
:1017D0002508F53B6300CA2BA603A536A40CA30C71
:1017E000A20CA61FCA2B21001710200021082100DF
:1017F0008C00200020082100990008002000E6014C
:10180000E701E801E90108007308E5007208E40057
:101810000134250824040319242CFA01FA0AA51B13
:10182000142CA435A50D0E2C25082702031D1A2CF7
:1018300024082602031C202C2408A6022508A73B06
:10184000A536A40CFA0B142C2708A5002608A40022
:101850000800D500043E8600870181105508043E2B
:1018600086000111F827003084318E248831200051
:10187000D601FF30E826883120001430D60A5602FF
:10188000031C392C84314F24883120000030AB01F7
:10189000AC01AD01AE01AF01AF0AF5248831D6002D
:1018A000560B422C0130AE01AD01AC00AA30AB00AA
:1018B0000830AF01AF0AF5248831D600D61B0034BA
:1018C0000030561D0130C4005508043E86008701D3
:1018D00001084406FE39440681003730AB01AC01F3
:1018E000AD01AE01AF01AF0AF5248831D600D61B99
:1018F00000340030561D0130C4005508043E8600F7
:101900008701C40DC40D01084406FB39440681005B
:10191000B801B80A5508043E8600010C890C01394B
:10192000F92688310038031DA22CB8015508043E61
:1019300086008701010C890C0139F92688310038AD
:10194000031900340930AB01AC01AD01AE01AF01A8
:10195000F5248831D600D61B00341030F500453010
:10196000F601F701F801F80AA42688312000D60014
:101970005608031D00344530F6005508043E860025
:1019800000308701011D013081314D21883155081A
:10199000860087017608C03F7708C13F7808C23FBC
:1019A0007908C33F5508043E860002308114AE0119
:1019B000AD01AC001030AB01AF01AF0AF5248831A6
:1019C000D6005608031D00343B30AB01AC01AD011D
:1019D000AE01AF01AF0AF5248831D6005608031DC9
:1019E0000034013084318E240134B000FF30E82609
:1019F00020002E08A3002D08A2002C08A1002B080F
:101A0000A000300883319323883184317C24200066
:101A1000B1000800210053082000D2002100540822
:101A20002000D300D401D5016608D2076708D33D52
:101A30006808D43D6908D53DD601D701CA01CB015C
:101A40002100520820004B02031D2A2D21005108BD
:101A500020004A02031800345508BF005408BE0095
:101A60005308BD005208BC005708C1005608C0000A
:101A70004E30C201C20AC300012688310038031962
:101A800000342000CE08031900344E08E53A03194B
:101A9000EB2D4E082E3A0319EB2D0130C402003015
:101AA000C53B440A0319450A031DEB2D46080319DB
:101AB0007E2D4E08053A03195F2D4E08602DE53046
:101AC000CC00CD014608860087014C0881005508EE
:101AD000BF005408BE005308BD005208BC005608A1
:101AE000013EC0000030573DC1000A30C200460A26
:101AF000C30001268831003803190034200048084B
:101B00000319992D5508BF005408BE005308BD00A5
:101B10005208BC0056080B3EC0000030573DC100C3
:101B2000C201C20A4808C3000126883100380319DF
:101B30000034200049080319C02D5508BF0054087F
:101B4000BE005308BD005208BC0056081A3EC00033
:101B50000030573DC1000230C2004E30C3000126A4
:101B600088310038031900344E30F201E9278831FA
:101B700020004908860087017208C03F7308C13FF2
:101B80004708031901345508BF005408BE00530824
:101B9000BD005208BC0056081C3EC0000030573D36
:101BA000C1000430C2004E30C30001268831003825
:101BB000031900344E30F201833145238831470840
:101BC000860087017208C03F7308C13F7408C23F96
:101BD0007508C33F01342030D6070318D70A5708C9
:101BE000023A5604031DFD2DD601D701D20A03196E
:101BF000D30A0319D40A0319D50ACA0A0319CB0A4E
:101C0000202D2100630820003F06031D172E210010
:101C1000620820003E06031D172E210061082000E7
:101C20003D06031D172E2100600820003C06031D01
:101C3000252E21005A0820004102031D232E2100D9
:101C400059082000400203186D2E2100600A031974
:101C5000610A0319620A0319630A031D332E452E14
:101C6000FF30E82688312100D90A0319DA0A59031E
:101C7000023003195A06031D302EF0268831FF303A
:101C80002100E300E200E100E00020003F08210025
:101C9000E30020003E082100E20020003D08210072
:101CA000E10020003C082100E00063082000B500AE
:101CB000210062082000B400210061082000B30068
:101CC000210060082000B200DB300320883100389A
:101CD000031900342100D901DA0120004108210054
:101CE0005A06031D772E20004008210059060319CB
:101CF000802ED90A0319DA0AFF30E82688316D2EC2
:101D0000200042082100D9070318DA0A2000C20384
:101D10004208FF3A0319962E43088600FF308701D8
:101D2000E826883181002000C30A862E21005A0847
:101D3000023A5904031D0134F026FF302100E3006C
:101D4000E200E100E0000134A00084317C2488310D
:101D50002000A100FE3A0319B82E2108080020082F
:101D60008600FF308701E826883181002000A00A24
:101D70000130F5020030F63B750A0319760A031D9F
:101D8000AF2E7708FF300319E02EE8268831F900DE
:101D9000FA01FA00F9017708860087017908C03F47
:101DA0007A08C13FFF30E8268831F900FA01770848
:101DB000860087017908810441317A088104E52E83
:101DC000E8268831FF30E8268831FF30E8260034E5
:101DD000F200720824009100141CEC2E1108080077
:101DE00020000C30AB01AC01AD01AE01AF01AF0A78
:101DF000F52CB900BA01BB01BE01BE0AB808031D2B
:101E0000062FC001C101C201C3010B2F4030C30026
:101E1000C201C101C001BA0A0319BB0A13303B0257
:101E2000893003193A0203180034B908031D262F1C
:101E30004308AE004208AD004108AC004008AB00CA
:101E40000130AF01AF0AF5248831322F4308B500C5
:101E50004208B4004108B3004008B2002930843180
:101E600030248831BC00BD01BF00BF1B00343E08D8
:101E700003193D2FC216BE010B2F3F1C01340B2F3F
:101E80006908BF006808BE006708BD006608BC009E
:101E90003630C0000430C101C200A030C3000126AA
:101EA000883100380319003421002008463A031D08
:101EB000652F2108413A031D652F2208543A031D5E
:101EC000652F2308313A0319672F8231322A200007
:101ED0006908BF006808BE006708BD006608BC004E
:101EE0000B30C0000D30C101C200A030C30001267C
:101EF0008831003803190034A030F201E927883115
:101F00007308023A7204031D0034210022082000E5
:101F1000ED000330F200A030E9278831730821007A
:101F2000D0007208CF000630F200A030E9278831D7
:101F30007308D2007208D1000B30F200A030E927FC
:101F40007308D8007208D7002508F200F30158087A
:101F5000F5005708F4008431672488317308D400F1
:101F60007208D3004F08D3075008D43DFF3020003B
:101F7000DE000130DF00E001E10121005108200016
:101F8000E200210052082000E3000530E401E501F1
:101F9000E235E30DE40DE50D890BC82F6208DE077D
:101FA0006308DF3D6408E03D6508E13D0930E13646
:101FB000E00CDF0CDE0C890BD72F5F082100CE0070
:101FC00020005E082100CD005308CD075408CE3D07
:101FD0000134F4007208F40774088600870174085D
:101FE000013E840085010008F3000108F2000800AA
:101FF0001530240092002A309500C030940008006B
:020000040001F9
:10E00000FF00FF00FF00FF00FF00FF00FF00FF0018
:10E01000FF00FF00FF00FF00FF00FF00FF00FF0008
:10E02000FF00FF00FF00FF00FF00FF00FF00FF00F8
:10E03000FF00FF00FF00FF00FF00FF00FF00FF00E8
:10E04000FF00FF00FF00FF00FF00FF00FF00FF00D8
:10E05000FF00FF00FF00FF00FF00FF00FF00FF00C8
:10E06000FF00FF00FF00FF00FF00FF00FF00FF00B8
:10E07000FF00FF00FF00FF00FF00FF00FF00FF00A8
:10E08000FF00FF00FF00FF00FF00FF00FF00FF0098
:10E09000FF00FF00FF00FF00FF00FF00FF00FF0088
:10E0A000FF00FF00FF00FF00FF00FF00FF00FF0078
:10E0B000FF00FF00FF00FF00FF00FF00FF00FF0068
:10E0C000FF00FF00FF00FF00FF00FF00FF00FF0058
:10E0D000FF00FF00FF00FF00FF00FF00FF00FF0048
:10E0E000FF00FF00FF00FF00FF00FF00FF00FF0038
:10E0F000FF00FF00FF00FF00FF00FF00FF00FF0028
:10E10000FF00FF00FF00FF00FF00FF00FF00FF0017
:10E11000FF00FF00FF00FF00FF00FF00FF00FF0007
:10E12000FF00FF00FF00FF00FF00FF00FF00FF00F7
:10E13000FF00FF00FF00FF00FF00FF00FF00FF00E7
:10E14000FF00FF00FF00FF00FF00FF00FF00FF00D7
:10E15000FF00FF00FF00FF00FF00FF00FF00FF00C7
:10E16000FF00FF00FF00FF00FF00FF00FF00FF00B7
:10E17000FF00FF00FF00FF00FF00FF00FF00FF00A7
:10E18000FF00FF00FF00FF00FF00FF00FF00FF0097
:10E19000FF00FF00FF00FF00FF00FF00FF00FF0087
:10E1A000FF00FF00FF00FF00FF00FF00FF00FF0077
:10E1B000FF00FF00FF00FF00FF00FF00FF00FF0067
:10E1C000FF00FF00FF00FF00FF00FF00FF00FF0057
:10E1D000FF00FF00FF00FF00FF00FF00FF00FF0047
:10E1E000FF00FF00FF00FF00FF00FF00FF00FF0037
:10E1F000FF00FF00FF00FF00FF00FF00FF00FF0027
:04000E00ACC9FFDE9C
:08000000FF3FFF3FFF3FFF3F00
:00000001FF
